:020000040000FA
:020000000528D1
:080008000900831603136830A0
:100010008F003F308500003086008030870026301A
:1000200006309F002430980019309900831603177A
:1000300088018901831203139030980087011A0800
:100040001A081A08860187011819292898183128D2
:100050003B28181218161A081A081A08071007154C
:100060003828181218161A081A081A0887100715BF
:100070009030980024288C1E2428071487141A080E
:10008000A000A01B52286A30200586000000000056
:1000900020088600000000006A30200586004030FD
:1000A0002005860005085520242883160313981C74
:1000B0005728831203139900080056006500720048
:1000C000730069006F006E00200036002F003100C1
:1000D00032002F00320030003000390020002D00A7
:1000E000200039003600300030002000620061003E
:0600F000750064007300BE
:02400E00D420BC
:02401000FF3E71
:00000001FF
